:020000040800F2
:10000000001000203D180008150300081703000821
:1000100000000000000000000000000000000000E0
:1000200000000000000000000000000019030008AC
:1000300000000000000000001B0300081D03000872
:100040008D1800088D1800088D1800088D180008FC
:100050008D180008B90300088D1800088D180008D5
:10006000000000008D1800088D1800088D18000889
:100070008D1800088D1800088D1800080000000079
:100080008D18000821030008000000008D180008EA
:100090008D1800087D0300088D1800088D180008D1
:1000A0008D1800088D1800088D1800088D1800089C
:1000B0008D18000800000000000000000000000093
:0C00C0008D180008000000008D180008DA
:1000CC0002B4714649084900095C49008E4402BCDF
:1000DC007047C04603B47146490840004900095EA8
:1000EC0049008E4403BC7047844608006146FFE714
:1000FC001FB503F08FF8002801D40021C8421FBDA2
:10010C0010B503F01DF84042013010BD10B503F0DE
:10011C0081F8002801DB002010BD012010BDC04675
:10012C0010B503F077F8002801DD002010BD012088
:10013C0010BDC04610B503F02BF8002801DC0020E0
:10014C0010BD012010BDC04610B503F021F80028E9
:10015C0001DA002010BD012010BDC0461C21012376
:10016C001B04984201D3000C10391B0A984201D38E
:10017C00000A08391B09984201D30009043902A26C
:10018C00105C40187047C0460403020201010101D3
:10019C00000000000000000040F2600040F260032C
:1001AC00C2F20000C2F2000310B5834205D040F247
:1001BC000003C0F2000303B1984710BD40F2600089
:1001CC0040F26003C2F20000C2F200031B1A9A1044
:1001DC00D90F8918491010B529B140F20003C0F2AB
:1001EC00000303B1984710BD10B540F26004C2F291
:1001FC000004237873B9FFF7CFFF40F20003C0F27D
:10020C0000032BB143F2A020C0F6000000E000BFB9
:10021C000123237010BDC04640F20003C0F200035E
:10022C0010B54BB140F2640143F2A020C2F20001C0
:10023C00C0F6000000E000BFFFF7C0FF10BDC046D5
:10024C0010B500F0CDF800F0D5F900F07FFA00F011
:10025C008DFA194801F03CFC184801F039FC16489D
:10026C0001F036FC40F2D07000F0DAF840F2E630E3
:10027C0000F0D6F8124C052000F0C4F9022000F072
:10028C00CFF821680F4801F0BFFB40F20323206830
:10029C0098420FD80C4C00F062FA0C4B01001880FD
:1002AC00200001F0B1FB00F0A9FA0100084801F0B0
:1002BC00ABFBDBE7074CEEE70A330008EA32000839
:1002CC00800000200C330008D03200087C00002095
:1002DC0019330008DE320008F8B50E0014000025B2
:1002EC0040F20777A54201DB2000F8BD715D05489F
:1002FC0001F091FA3900034801F091FA0028F9D085
:10030C000135EFE700380140FEE7FEE7FEE7FEE7C8
:10031C007047000070B50121134800F0DEFF0400A7
:10032C00012816D1114D01000F4800F0E1FF2B7888
:10033C0083B1902040F200210022C00500F0B4FCF3
:10034C0044F60031084800F0C0FF2B785A42534164
:10035C002B7070BD902040F200212200C00500F0EF
:10036C00A3FC40F22031EDE7001000407E0000209D
:10037C0010B501210B4800F0B0FF0400012810D18A
:10038C000100084800F0B4FF200000F025FC00211B
:10039C00054800F09CFF044800F088FF014800F07D
:1003AC008AFF10BD004401400048014010B50120F7
:1003BC0000F032FC040001280DD100F031FC0021CA
:1003CC00054801F0B9F9054B1860034800F073FFBC
:1003DC00200000F009FC10BD004801408000002006
:1003EC00052010B5404200F0A5FD084B186802F03E
:1003FC0067FE074902F02EFA064B07491860186889
:10040C0002F03AFB054B186010BDC04600000020FE
:10041C000024F44A8800002000007A448400002064
:10042C000D4B10B51C6802F04BFE211C02F024FB96
:10043C0002F0F8F90022094B094958609A60013220
:10044C001A601A680A40012AFBD001211A688A43F3
:10045C001A6000229A6010BD8400002010E000E0B9
:10046C000100010030B5902440F2002585B0E40570
:10047C0040F2115000F06CFD2B00200000220121F5
:10048C0000F0D4FB2B0020000322002100F0EEFB37
:10049C00012229002000144C00F006FC40F20470EC
:1004AC0000F056FD200000F051FE684600F0A8FE5A
:1004BC0041F61F430025009340F2E73369462000C4
:1004CC000293019500F0A4FE200000F0F9FE01213A
:1004DC00200000F0FEFE200000F0E8FE29001120B4
:1004EC0000F0EAFC05B030BD0010004010B59024BF
:1004FC0040F2115000F02CFDE40540F20E6000F0CB
:10050C0027FD20000C22012100F0D3FB20000C233E
:10051C000122022100F08AFB20000D4C0C23012249
:10052C00002100F0A3FB200001F01AF9E1212000CA
:10053C00490201F031F92000042101F064F908218D
:10054C00200001F058F9200001F050F910BDC04610
:10055C000038014070B540F2125088B000F0F8FC41
:10056C000223224C19002000002200F05FFB022322
:10057C0020000322002100F079FB02220021200040
:10058C001B4C00F096FB40F2087000F0E1FC2000E0
:10059C0000F0DCFD04A800F033FE0025EF2301265B
:1005AC0004A9200006930495059500F031FE01A8DE
:1005BC0000F0A1FE2900200001AA019602950395E6
:1005CC0000F0A2FE29002000782200F0D7FF602264
:1005DC002900200000F0A8FF200000F071FE31007F
:1005EC00200000F076FE08B070BDC0460004004844
:1005FC000020004010B5FFF735FFFFF777FFFFF73E
:10060C00A9FF10BD70B5782200210400104800F03D
:10061C00B5FF702200210E4800F086FF0C4800F058
:10062C0045FE0C4800F042FE0025A54203D10848C7
:10063C0000F041FE70BD0121054800F04EFE00287F
:10064C00F9D00121024800F053FE0135EDE7C04618
:10065C00002000400044014030B5134D85B004002B
:10066C0040F2116000F074FC280000F06FFD684649
:10067C0000F0C6FD47236A46009300236946280014
:10068C00013C01931373029400F0C2FD280000F0AA
:10069C0017FE2800012100F01CFE0121152000F09E
:1006AC000BFC05B030BDC0460044014010B540F213
:1006BC00115000F04DFC40F2006000F049FC0022AB
:1006CC00902001231100C00500F0B0FA0021052094
:1006DC0000F0F2FB0021080000F012FD01220021C5
:1006EC00100000F03DFA012000F090FA10BD00005F
:1006FC0070B5144D86B040F2126000F029FC02ACCB
:10070C00280000F023FD200000F07AFD472300268E
:10071C0002934EF65F232100280004930396267360
:10072C0000F076FD684600F03AFF074B6A460093EE
:10073C00C02331009B022800019300F061FF06B03A
:10074C0070BDC046004801400A00020010B5FA20F6
:10075C00FFF782FFFFF7AAFFFFF7CAFF10BD1123B7
:10076C00584341F29A03C01880B2704710B540F25A
:10077C0016501F4C00F0ECFB40F2157000F0E8FB3B
:10078C0020000222012100F094FA01222000110025
:10079C0000F08FFA022320001900012200F046FA23
:1007AC00200002230322012100F060FA0123200023
:1007BC001A00022100F03AFA012320000D4C190016
:1007CC00032200F053FA200000220B4900F0A0FA9B
:1007DC000022B4231100200000F020FB200000F0C8
:1007EC003BFB40F20041200000F024FB10BDC04652
:1007FC000014004800540040A0860100F8B540F2F7
:10080C0000417E4800F016FB002540F201663100E5
:10081C007A4800F037FB41F28833040050B19D4216
:10082C0005D1774801F054F94EF6FC70F8BD01354E
:10083C00ADB2ECE79D42F4D0704800F012FB40F2F0
:10084C00005529006D4800F01DFB41F2883320B99A
:10085C009C42E9D00134A4B2F3E79C42E4D00222DA
:10086C00B4216648524200F0EDFA002440F20155E2
:10087C002900624800F006FB41F2883320B99C4203
:10088C00D2D00134A4B2F3E79C42CDD040F2015156
:10089C005A4800F000FB002440F207552900574845
:1008AC0000F0F0FA41F2883320B99C42BCD00134FC
:1008BC00A4B2F3E79C42B7D00721504800F0DDFA10
:1008CC00002540F2025631004C4800F0DBFA41F2B0
:1008DC008833040020B19D42A6D00135ADB2F2E7B9
:1008EC009D42A1D0454800F0BCFA40F200552900C9
:1008FC00424800F0C7FA41F2883328B99C4200D133
:10090C0092E70134A4B2F2E79C4200D18CE70122B9
:10091C00B4213A4800F096FA002440F2015529001F
:10092C00364800F0AFFA41F2883328B99C4200D126
:10093C007AE70134A4B2F2E79C4200D174E740F2AA
:10094C0001512E4800F0A7FA002440F20655290068
:10095C002A4800F097FA41F2883328B99C4200D11A
:10096C0062E70134A4B2F2E79C4200D15CE7234871
:10097C0000F085FA0024050040F2065631001F48AD
:10098C0000F080FA41F2883328B99C4200D14BE741
:10099C000134A4B2F2E79C4200D145E7174800F0BD
:1009AC006EFA00210400154800F044FA002640F2CB
:1009BC0006573900114800F065FA41F2883328B91E
:1009CC009E4200D130E70136B6B2F2E79E4200D12A
:1009DC002AE70A4800F053FA084800F048FA2302C4
:1009EC009BB2084A2B435B009B1842F23412181C32
:1009FC009BB2934200D9101C80B217E70054004000
:100A0C00223300084D95FFFF012337B5464A116884
:100A1C000B431360022311681942FCD08021434B15
:100A2C001868014319600021019101997F2943D96C
:100A3C0090211868014319600021019101997F29C7
:100A4C003DD903200F241968814319601168384877
:100A5C00014011601968374801401960196836481F
:100A6C000140364819600168A14301603449354C96
:100A7C000868204008600868334C2040086008680B
:100A8C00324C4000400808600121206888432060F7
:100A9C0000242F480460106801431160022040F2CA
:100AAC0000511468044202D101390029F9D1022104
:100ABC001068084206D1FEE701990131B4E70199AB
:100ACC000131BAE70725234C2068A8430143216074
:100ADC001968214819601968196019681960196832
:100AEC000140196018681D49014319608021106884
:100AFC004904014311608021890410680842FCD02C
:100B0C0003211A688A431A60022219680A430C21CD
:100B1C001A601A680A40082AFBD1802000210005BF
:100B2C0000F0FCF937BDC046001002400410024032
:100B3C00FFFFF2FE0C00FF08FFFFC2772C100240F3
:100B4C0030100240FCFEFFFFFFFFFEFF341002409E
:100B5C000810024000200240FFFFC2F7000004080A
:100B6C00F7B5194E194D33680191834333602B68E7
:100B7C00174C83432B602368C74383432360154B77
:100B8C00196881431960019969B101290FD0012AB3
:100B9C0011D0022A15D02AB92268024322601A68A1
:100BAC003A401A60F7BD316801433160EFE72968BC
:100BBC0001432960EBE722683A4022601A6802433D
:100BCC00EFE722680243F8E7000401400404014007
:100BDC00080401400C040140024A136803431360EB
:100BEC007047C04600040140024A136883431360F7
:100BFC007047C04600040140034B1B681840431E5D
:100C0C009841C0B27047C04614040140014B1860B3
:100C1C007047C0461404014010B5FFF7EDFF10BD3E
:100C2C00014B18607047C04614040140F0B585B004
:100C3C00019103270021029203930268C3680124E7
:100C4C008C40039D25420AD03D004C00A540019EDE
:100C5C00AA43AB43029DA640A54032432B4301312E
:100C6C001029ECD10260C36005B0F0BDF7B501925C
:100C7C00012916D14168194300240126032741603C
:100C8C0081683500A5402B4206D03A006500AA4089
:100C9C009143019AAA4011430134102CF1D1816087
:100CAC00F7BD41689943E7E70AB1816170478162FA
:100CBC00FCE7F7B5002401260F270091016A436A6F
:100CCC0001923500A540019A2A4206D03A00A500AF
:100CDC00AA409143009AAA4011430134082CF0D148
:100CEC00002401260F27250032000835AA401500E4
:100CFC00019A2A4206D03A00A500AA409343009AD2
:100D0C00AA4013430134082CEDD101624362F7BDB4
:100D1C00F8B5040002200D0016007F2700F03CF906
:100D2C00394A3A490300B0FBF2F238008B4200D842
:100D3C0010006168B9430143616035498D4214D894
:100D4C0001327E2A0CD927626D00B3FBF5F0E26903
:100D5C00042800D204200005000D1043E061F8BD0A
:100D6C00022A00D802222262EEE72A4A40F2E83137
:100D7C00954225D840F22C124243B2FBF1F20132DB
:100D8C002262A6B903206843234AB3FBF0F0E3695F
:100D9C001340E36103050BB90133184348F2000318
:100DAC00E2691343E361E3690343E361D7E7192085
:100DBC006843B3FBF0F044F20003E2691343E8E745
:100DCC0078224243B2FBF1F2013222629EB9032235
:100DDC006A431149B3FBF2F2E3690B40E36148F259
:100DEC000003E1690B43E361E3691343E36101230E
:100DFC0090342360B3E719226A43B3FBF2F244F256
:100E0C000003E1690B43E9E740420F00BFDD9107A6
:100E1C00A0860100801A0600FFBFFFFF30B5022537
:100E2C0004689B05AC439B0D0C4313430460836027
:100E3C0030BD00000368024A13400B430360704747
:100E4C00FFFBFFFF10B5012423000B43023201D13D
:100E5C000B00A343036110BD01230268134303601D
:100E6C00704740F20013026813430360704740F26E
:100E7C0000230268134303607047016170470069E7
:100E8C00C0B270478B091B1818681F231940C84043
:100E9C001E3B1840704740F20153994202D14369FE
:100EAC00836970478B091B181F2001401E3888402E
:100EBC001A6882431A60F4E730B5FF24032223003A
:100ECC000240D200934089012140914042B2DB4361
:100EDC00002A12DB40F200350E4C820892001219E7
:100EEC00545923400B431F215351012201408A4086
:100EFC00430908499B005A5030BD0F221040083856
:100F0C00054A800880008018C26913400B43C361F6
:100F1C00F2E7C04600E100E000ED00E0034B1940B1
:100F2C00034B01439960BFF34F8F704780FFFF1F46
:100F3C0000ED00E0054B1A68042802D1104318603C
:100F4C00704704218A431A60FAE7C04610E000E0BB
:100F5C00054B8209D2181F2318401E3B8340116891
:100F6C000B4313607047C046001002401F218309D9
:100F7C0008401E398140034A9B181A688A431A603C
:100F8C007047C0460010024010B5FFF7E1FF10BDDE
:100F9C0010B5FFF7EBFF10BD70B5524E88B004AD25
:100FAC003100102210360400280000F0F6FE082252
:100FBC003100684600F0F1FE0822310002A800F072
:100FCC00ECFE0C21484A13680B40082B36D11168F3
:100FDC0013688902090F1B0129D50B001133116805
:100FEC00C90329D50F204149096801404048013106
:100FFC00B0FBF1F14B43180011686E460906090F5E
:10100C00695C0725C84001001068000A2840365C5E
:10101C001068C00A284002AD285C0D00C540052CA4
:10102C0058D82000FFF74CF80D0C10581340102323
:10103C000F29D4D08B1CD2E72E49DBE72C4BDAE7F7
:10104C000B00180008B070BD0B00F340F9E72A48FC
:10105C000368DB0506D40368284ADB03DB1713405F
:10106C009B18EEE7032312680068920B1A40C00F1E
:10107C00022A0DD09A4212D0012A02D028B96B084C
:10108C00DFE7AB080028DCD00523B1FBF3F3D8E78E
:10109C0018B90623B5FBF3F3D3E70723F5E7EB0801
:1010AC000028CED00923F0E7032213490868104228
:1010BC0012D0086810400128C3D00B681340022BD3
:1010CC000CD00B681340033B5A425341084A5B4215
:1010DC001340B6E70023B4E72B00B2E748F2000355
:1010EC00AFE7C046B8320008041002402C10024092
:1010FC0000127A0000093D0030100240809FD5009C
:10110C0010B503240F230C40A4000200A340A240FE
:10111C00DB4388080F290AD8FEF7D2FF020A0C0E0F
:10112C000649086803400B600B6813430B6010BD45
:10113C000349F6E70349F4E70349F2E708000140E5
:10114C000C0001401000014014000140254B10B56B
:10115C0098421AD009D8244B984226D0234B984257
:10116C002AD0234B984219D010BD224B98422AD03A
:10117C00214B98422ED0214B9842F5D140F21030A1
:10118C00FFF702FF40F2103005E040F20B30FFF7A2
:10119C00FBFE40F20B30FFF7FBFEE5E740F20140AF
:1011AC00FFF7F2FE40F20140F5E740F20440FFF792
:1011BC00EBFE40F20440EEE740F20840FFF7E4FE9D
:1011CC0040F20840E7E740F21130FFF7DDFE40F255
:1011DC001130E0E740F21230FFF7D6FE40F2123049
:1011EC00D9E7C046002C0140001000400020004010
:1011FC000004004000440140004801400040014010
:10120C0000234FF6FF7203604360826003737047E4
:10121C000B8810B583621E4B984202D01D4A904237
:10122C000BD170240268A243026004684A882243EE
:10123C00026004688A88224302608A68C26298420B
:10124C000DD0144A90420AD0134A904207D0134A48
:10125C00134C0240A24202D0124A904213D10268AF
:10126C00114C224002600468CA88224302609842F2
:10127C0007D00A4B0A4A0340934202D0094B9842CA
:10128C0001D10B7B0363012342691343436110BDFE
:10129C00002C01400004004000200040FFFBFFFF39
:1012AC000040014000480140FFFCFFFF01230268A1
:1012BC001343036070470122036893430360704734
:1012CC0080230268134303607047C1627047416218
:1012DC007047C3680B43C3607047C268036908005A
:1012EC001840194203D011404B1E9941C8B27047A7
:1012FC00C943016170470023038043808380C3800E
:10130C000381438170470000030030B508000329B6
:10131C0042D81188764CFEF7D3FE02408CCA0125C8
:10132C00186AA843186298690235A8439861186A2C
:10133C00014302201962196A81431962186A918863
:10134C0001431962A34207D06A496B481940814294
:10135C0002D06A498B421FD10420196A8143196259
:10136C00186A5188014308201962196A814319626D
:10137C00186AD18801431962596861480140596063
:10138C00586811890143596059685E480140596099
:10139C00596852890A435A6030BD1025186A0901F0
:1013AC00A84318629869584D28409861186A0143FF
:1013BC0020201962196A814319629188186A0901FF
:1013CC0001431962A34226D14020504B1968814336
:1013DC001960518818680901014380201960196847
:1013EC0081431960D1881868090101431960484B81
:1013FC004048196801401960118918688900014337
:10140C0019601968434801401960528919689200A3
:10141C000A431A60C0E738498B42BDD13E49354872
:10142C000B6803400B60138908689B0003430B6037
:10143C00B2E7186A324D090228401862D86905359E
:10144C00FF35A843D861186A01431962196A2D48FF
:10145C00014019629188186A090201431962A3427A
:10146C0000D099E7294B234819680140196051882D
:10147C00186809020143196019682648014019606F
:10148C00D1881868090201431960214B2348196857
:10149C000140196011891868090101431960196824
:1014AC001F4801401960528919681201B0E7186A87
:1014BC001A4D090328401862D869134D2840D86189
:1014CC00186A01431962196A15480140196291881A
:1014DC00186A090301431962A34200D05CE70C4966
:1014EC0010480B6803400B60138908689B019DE74B
:1014FC00002C0140FFFBFFFF004001400048014071
:10150C00FFFEFFFFFFFDFFFFFFFCFFFF202C014054
:10151C00042C0140FFF7FFFF04400140FFEFFFFFE9
:10152C00FFDFFFFFFFBFFFFF030000B5080003292B
:10153C000AD8FEF7C5FD020A11197020996981437A
:10154C00996199690A439A6100BD99690A48120226
:10155C00014099619969F5E77020D9698143D96196
:10156C00D9690A43DA61EFE7D969034812020140ED
:10157C00D961D969F5E7C046FF8FFFFF030000B5BD
:10158C000800032904D8FEF79BFD020406085A63E1
:10159C0000BD9A63FCE7DA63FAE71A64F8E7002304
:1015AC000122038042808380C3807047030000B512
:1015BC00080003290AD8FEF783FD020A11190C2032
:1015CC0099698143996199690A439A6100BD996946
:1015DC000A481202014099619969F5E70C20D96912
:1015EC008143D961D9690A43DA61EFE7D9690348C4
:1015FC0012020140D961D969F5E7C046FFF3FFFF3C
:10160C00030070B5032924D808001488FEF758FD90
:10161C000226436601250A26186AA8431862186A2E
:10162C00B0431862186A2043032418629869A043D7
:10163C0098619C6950882043F02498619869A04374
:10164C009861D0889C69000120439861186A054311
:10165C001D6218009288FFF7A9FF70BD1025A02607
:10166C00186A2401A8431862186AB0431862186AF1
:10167C0004431C6298692A4C2040986150889C69EC
:10168C000002204398619869264C20409861D088CC
:10169C009C690003D8E7186A234D2402284018627D
:1016AC00186A224D28401862186A04431C620324ED
:1016BC00D869A043D861DC6950882043F024D861F4
:1016CC00D869A043D861D088DC6900012043D86177
:1016DC0040F200101C6A20431862BAE7186A144DD5
:1016EC00240328401862186A124D28401862186AA0
:1016FC0004431C62D8690A4C2040D8615088DC69CC
:10170C0000022043D861D869064C2040D861D088AB
:10171C00DC6900032043D8611C6A41F20000DAE75F
:10172C00FFFCFFFFFF0FFFFFFFFEFFFFFFF5FFFFBB
:10173C00FFEFFFFFFF5FFFFF03000022080000B573
:10174C00032904D8FEF7BCFC020507095A6B1000EC
:10175C0000BD9A6BFBE7DA6BF9E71A6CF7E7000050
:10176C000B4B10B598420BD00A4B984207D140F264
:10177C000E30FFF709FC40F20E30FFF709FC10BDEC
:10178C0040F21140FFF700FC40F21140F5E7C04673
:10179C000044004000380140124B70B504000D00AD
:1017AC00984216D0104B00209C4202D10530FFF716
:1017BC00F3FB22686B0812040DD54100C918B1FB6C
:1017CC00F5F14FF6F0720B075B0F11400B43E36022
:1017DC0070BD0220EBE7C018B0FBF5F189B2E160F7
:1017EC00F6E7C0460044004000380140012302687F
:1017FC001343036070470822036893430360036834
:10180C000B4303607047042203689343036003682F
:10181C000B4303607047C905C90D816270478B0982
:10182C001B1818681F231940C8401E3B18407047EE
:10183C000D488546002103E00C4B5B5843500431A6
:10184C000B480C4B42189A42F6D30B4A02E0002389
:10185C0013600432094B9A42F9D3FFF7D5F800F024
:10186C0071FAFEF7EDFCFEE700100020E0330008F3
:10187C00000000206000002060000020DC0100203F
:10188C00FEE70000002310B5040003604360836092
:10189C0081814366C281036143618361190008221F
:1018AC005C3000F001FA0B4B246263620A4BA362BA
:1018BC000A4BE3620A4B23630A4B9C4205D00A4B4A
:1018CC009C4202D0094B9C4203D12000583000F0BE
:1018DC0061FA10BDF11A0008191B0008511B000811
:1018EC007D1B00088C000020F40000205C0100200F
:1018FC0010B5034A0349044800F06AF810BDC0460D
:10190C0004000020152600081400002041680B4B31
:10191C0010B50400994201D000F076FEA168084B86
:10192C00994202D0200000F06FFEE168054B99420D
:10193C0002D0200000F068FE10BDC0468C000020D4
:10194C00F40000205C01002010B5094B094A042169
:10195C001A6009480022FFF795FF01220921074868
:10196C00FFF790FF022212210548FFF78BFF10BDF5
:10197C00C4010020FD1800088C000020F400002099
:10198C005C01002010B5024800F005FA10BDC046FD
:10199C00CD01002010B5024800F0FEF910BDC04684
:1019AC00CD01002010B50400FFF7ECFF236A13B142
:1019BC00FFF7F0FF10BD044B2362044B1B68002B98
:1019CC00F6D1FFF7C1FFF3E719190008C401002095
:1019DC00F7B51400002600900191A5686768013FD7
:1019EC0004D52468002CF8D13000FEBDAB89012B46
:1019FC0008D90E22AB5E013304D029000098019B5C
:101A0C00984706436835EAE70FB407B5054904ABB8
:101A1C00086804CB8168019300F0EAFA03B008BCB3
:101A2C0004B0184710000020036A70B505000E00C2
:101A3C0084680BB9FFF7B6FF636EDB0705D4A38987
:101A4C009B0502D4A06D00F0A6F9A3891B0701D554
:101A5C002369F3B92100280000F0CEF8C8B10125A4
:101A6C006D42636EDB0705D4A3899B0502D4A06D80
:101A7C0000F092F9280070BD0136A360002B04DA47
:101A8C00A2699A4216DC0A2914D023685A1C2260D7
:101A9C001970A3683178013B0029EDD1A360002BAC
:101AAC000FDA220028000A3100F068F80130D6D095
:101ABC000A25D6E72200280000F060F80130E8D1B2
:101ACC00CDE723685A1C22600A221A70F0E7000046
:101ADC0010B5034B01001868FFF7A6FF10BDC046F8
:101AEC001000002070B50C000E25495F00F006F9BF
:101AFC00002803DB636D1B18636570BDA389024A64
:101B0C001340A381F9E7C046FFEFFFFFF8B51F00B4
:101B1C008B8905000C001600DB0505D50E23C95E6C
:101B2C000022022300F0D8F8A389054A28001340AC
:101B3C00A38132000E23E15E3B0000F0F1F8F8BD0A
:101B4C00FFEFFFFF70B50C000E25495F00F0C4F8E5
:101B5C00A389421C03D1054A1340A38170BD41F2F5
:101B6C0000021343A3816065F8E7C046FFEFFFFF57
:101B7C0010B50E23C95E00F09FF810BDF8B5060035
:101B8C000D00140018B1036A0BB9FFF70BFFA36922
:101B9C00A360A3891B0701D5236943B92100300039
:101BAC0000F02AF818B101256D422800F8BD236910
:101BBC002068EFB2C01A6369EDB2834205DC2100E4
:101BCC00300000F021FD0028EDD1A3680130013B6D
:101BDC00A36023685A1C22601F706369834204D07F
:101BEC00A389DB07E1D50A2DDFD12100300000F0FD
:101BFC000BFD0028D9D0D6E72A4B70B50500186824
:101C0C000C0018B1036A0BB9FFF7CCFE0C22A35ED3
:101C1C001A0722D4DA0607D409222A6040220120AE
:101C2C001343A381404237E05B0712D5616B41B18E
:101C3C0023004433994202D0280000F0B7F8002367
:101C4C0063632422A3899343A381002363602369E4
:101C5C0023600823A2891343A38123695BB940F253
:101C6C00802140F20022A3890B40934203D0210033
:101C7C00280000F01BFD0C22A35E01211A000A4073
:101C8C000B420AD00022A26062695242A261226910
:101C9C0000200AB91A06C1D470BD990700D4626934
:101CAC00A260F4E71000002003008218934200D1D8
:101CBC00704719700133F9E7002370B5054D040026
:101CCC0008002B6000F06EFD431C02D12B6803B1A1
:101CDC00236070BDC801002070B50400080011001D
:101CEC001A000023044D2B6000F078FD431C02D138
:101CFC002B6803B1236070BDC801002070B50400CF
:101D0C00080011001A000023044D2B6000F070FD38
:101D1C00431C02D12B6803B1236070BDC8010020A5
:101D2C0070B50400080011001A000023044D2B604C
:101D3C00FEF7D2FA431C02D12B6803B1236070BDAD
:101D4C00C801002070B500250E4C0F4BE41AA410EE
:101D5C00A54209D1002501F09DFA0C4C0C4BE41A5C
:101D6C00A410A54207D170BD074AAB009B181B6895
:101D7C0098470135ECE7064AAB009B181B6898475F
:101D8C000135EEE7D8330008D8330008DC330008FF
:101D9C00D8330008704770477047002310B59A423B
:101DAC0000D110BDCC5CC4540133F8E770B505000C
:101DBC000C0079B1043C2368002B00DAE4182800ED
:101DCC0000F0DEF81C4A13682BB96360146028001D
:101DDC0000F0DEF870BDA34208D9206821188B42B0
:101DEC00F3D119685B6809182160EEE71A005B688B
:101DFC000BB1A342FAD911685018A0420BD120683C
:101E0C000918501811608342E1D118685B684118B9
:101E1C0011605360DBE7A04202D90C232B60D6E79C
:101E2C00206821188B4203D119685B68091821605E
:101E3C0063605460CBE7C046D401002070B50F4EF0
:101E4C000D003168040011B900F090FC30602900DD
:101E5C00200000F08BFC431C03D101256D422800AF
:101E6C0070BD0323C51C9D43A842F8D0291A20003D
:101E7C0000F07CFC0130F2D1EFE7C046D00100202D
:101E8C00F7B50322CB1C9343083305001F000C2B22
:101E9C0034D20C27B94233D8384E280000F070F8F1
:101EAC0033681C00002C2FD139002800FFF7C6FF27
:101EBC000400431C5FD134680094009B002B4AD172
:101ECC00002C52D023682800E3180099019300F0ED
:101EDC004DFC019B834248D123682800FF1A39002E
:101EEC00FFF7ACFF013040D02368DB192360336867
:101EFC005A68002A33D1009B336019E0002BC9DAF1
:101F0C000C232B600020FEBD2168C91B20D40B299B
:101F1C000AD9E2192760A34204D1326063681160C8
:101F2C00536005E05A60F9E76268A3420ED1326053
:101F3C00280000F02DF8200007220B30231D9043C1
:101F4C00C21A9842DFD01B1AA350DCE75A60EFE7A5
:101F5C0023006468A6E7009C63680093ADE71A0051
:101F6C005B68A342FBD10023DAE70C2328002B602B
:101F7C0000F00EF8C6E70760DAE7C046D40100208F
:101F8C0010B50248FFF707FF10BDC046CC0100207A
:101F9C0010B50248FFF700FF10BDC046CC01002071
:101FAC00936810B5013B9360002B04DA9469A3424B
:101FBC0007DB0A2905D01368581C1060197008003B
:101FCC0010BDFFF7DBFD0100F9E7F8B506000F00C7
:101FDC001400D518AC4201D1002007E021783A005A
:101FEC003000FFF7DDFF0134431CF3D1F8BD0000D6
:101FFC00F0B5A1B00D0017001E00039018B1036AD4
:10200C000BB9FFF7CFFC6B6EDB0705D4AB899B05D7
:10201C0002D4A86DFFF7BFFEAB891B0701D52B6956
:10202C0093B929000398FFF7E7FD68B16B6EDB07E6
:10203C0003D50120404221B0F0BDAB899B05F8D4FB
:10204C00A86DFFF7A9FEF4E7002308AC6361203309
:10205C0063761033A37607963E0033780BB1252BAD
:10206C0046D1F31B0593BE420BD03A0029000398CE
:10207C00FFF7ABFF013000D1AEE06369059A9B1806
:10208C0063613378002B00D1A6E001220023524279
:10209C00626004A954325218771C2360E360A36079
:1020AC001370A36505223978574800F06FFB7E1C2E
:1020BC0000BB2268D30604D5532304A95B18202146
:1020CC001970130704D5532304A95B182B2119701D
:1020DC003B782A2B17D03E00002140F20A0C012736
:1020EC00E3683278701C303A092A4DD989B917E067
:1020FC000136B2E7444B2268C01A012383401343D4
:10210C0037002360CEE7079B191D1B680791002B36
:10211C0001DB0B9304E05B42E36002231343236077
:10212C0033782E2B0CD173782A2B33D1079B0236A4
:10213C001A1D1B680792002B01DA01235B420993DD
:10214C00324F03223800317800F020FB30B14023AD
:10215C00C01B83402268013613432360317806226A
:10216C002B48771C217600F011FB002843D0294B1B
:10217C0033BB0722079B07339343083307936369E9
:10218C00049A9B18636167E761464B43060039006C
:10219C009B18A6E7002340F20A0C1A00012701360F
:1021AC0063603178701C3039092903D9002BC7D0F2
:1021BC000992C5E763465A4306003B005218F0E704
:1021CC0007AB00932A002100134B039800E000BFDB
:1021DC000490049B0133D2D16B6EDB0705D4AB8921
:1021EC009B0502D4A86DFFF7D7FDAB895B0600D524
:1021FC001FE70D981FE707AB00932A002100064B41
:10220C00039800F079F8E3E7273300082D33000832
:10221C003133000800000000D71F0008F7B5160086
:10222C0001938A680B690C000090934200DA13004A
:10223C0022003360433212780AB1013333602368D1
:10224C009B0602D5336802333360226806231500DF
:10225C001D401A4227D0230043331B785A1E93414A
:10226C002268920630D4220001990098089D4332CE
:10227C00A847013025D00622236800251340042BE3
:10228C0005D13368E568ED1AEB43DB171D40A368F5
:10229C002269934201DD9B1AED180026B54220D12C
:1022AC00002010E00135E36832689B1AAB42D2DDA6
:1022BC002200012301990098089F1932B847013078
:1022CC00F0D101204042FEBD3020E11843310870AE
:1022DC0021005A1C45310978A2184332023311707F
:1022EC00C1E72200012301990098089F1A32B847D0
:1022FC000130E6D00136D1E7F0B50E0089B004927A
:10230C00039005930C00097E0E9A4336782907D862
:10231C00622909D8002900D1B7E0582900D1A0E0E2
:10232C0025004235297022E0080063381528F7D8BB
:10233C00FDF7D0FE16001F00F6FFF6FFF6FFF6FFC6
:10234C001F00F6FFF6FFF6FFF6FF9E003400430079
:10235C00F6FFF6FFAF00F6FF3400F6FFF6FF47007E
:10236C00250013684235191D1B6811602B70012361
:10237C009CE013682068191D050609D51B681160BF
:10238C00002B02DA2D225B4232700A225B4832E0CB
:10239C001B6811604006F3D51BB2F1E71068256885
:1023AC0008C82F0602D46D0600D59BB21060082217
:1023BC0052486F291BD00A2219E0202321680B43B5
:1023CC00236078214E482300453319701568216825
:1023DC0008CD0F0602D44F0600D59BB21560CA0774
:1023EC0002D520220A432260002B3CD0102221006F
:1023FC00002543310D706168A160002908DB40F2B3
:10240C00040C674625681943BD432560350061B14E
:10241C003500B3FBF2FC61465143591A415C013D56
:10242C002970190063468A42F3D9082A09D1236816
:10243C00DB0706D5626823699A4202DC3023013D32
:10244C002B70761B2661059B210000930398049B3F
:10245C0007AAFFF7E3FE01302CD10120404209B05E
:10246C00F0BD2648AFE7202122688A432260BDE7F1
:10247C0013682568181D616910601B682F0601D54B
:10248C00196002E06D06FBD519800023350023612D
:10249C00D9E71368191D11601D68002128006268B6
:1024AC0000F074F908B1401B60606368236100237D
:1024BC003370C8E72A00236904990398059DA8473F
:1024CC000130CAD023689B0715D4079BE06898425B
:1024DC00C5DA1800C3E72200012304990398059E6E
:1024EC001932B0470130B8D00135E368079A9B1A0E
:1024FC00AB42F0DCE9E70025F7E7C04638330008CB
:10250C0049330008F7B50C228B5E05000C001A0746
:10251C0053D44A68002A02DC0A6C002A4BDDE76AB5
:10252C00002F48D0002241F200002E682A601A00C9
:10253C00216A0240034230D0626DA3895B0705D546
:10254C006368D21A636B0BB1236CD21A0023280078
:10255C00E76A216AB847A289431C06D129681D295C
:10256C0044D8284BCB40DB0740D50023636023695C
:10257C002360D20404D5431C01D12B6803B96065D8
:10258C00616B2E60B9B123004433994202D028000C
:10259C00FFF70CFC002363630DE001232800B84710
:1025AC000200431CC9D12B68002BC6D01D2B01D0B7
:1025BC00162B1AD12E6000201EE00E69002EFAD0C8
:1025CC000F680E60BA1B019200229B0700D14A696A
:1025DC00A260019B002BEEDDA36A32001F002800D5
:1025EC00019B216AB847002807DCA28940230120FF
:1025FC0013431BB2A3814042FEBD019B36181B1A2C
:10260C000193E6E7010040200B6970B505000C0052
:10261C0013B90025280070BD18B1036A0BB9FFF778
:10262C00C1F90C22A35E002BF3D0626ED20704D446
:10263C009B0502D4A06DFFF7AEFB28002100FFF72D
:10264C0061FF636E0500DB07E4D4A3899B05E1D42D
:10265C00A06DFFF7A1FBDDE770B50E001D000E238A
:10266C00C95E140096B000290CDAB28980231100DF
:10267C0019401A4214D140F2004300202960236013
:10268C0016B070BD6A4600F04FF80028EDDB4FF233
:10269C00000301991940044BC9184B425941EAE710
:1026AC0000214023E9E7C04600E0FFFFF0B5022619
:1026BC008B8905000C0085B0334207D023004733CB
:1026CC00236023610123636105B0F0BD03AB02AA53
:1026DC00FFF7C2FF029F019039002800FFF7D0FBE3
:1026EC0040B90C22A35E9A05EED4032293431E43F9
:1026FC00A681E3E78023A28920601343A381039B77
:10270C00206167615BB128000E23E15E00F01EF8CA
:10271C0028B10323A2899A43023B1343A381A389C3
:10272C00019A1343A381CFE7002370B5064D040033
:10273C00080011002B6000F03FF8431C02D12B68FD
:10274C0003B1236070BDC046C8010020002370B5E2
:10275C00054D040008002B6000F038F8431C02D132
:10276C002B6803B1236070BDC8010020002370B535
:10277C00054D040008002B6000F044F8431C02D106
:10278C002B6803B1236070BDC8010020C9B2821848
:10279C00904201D10020704703788B42FBD001306E
:1027AC00F6E7000040F2C81358220120C2F20003E1
:1027BC0040421A607047C04640F2C81358220120AC
:1027CC00C2F2000340421A607047C04640F2C81380
:1027DC005822C2F2000300201A60704740F2C8135E
:1027EC0058220120C2F2000340421A607047C046D2
:1027FC0040F2C81358220120C2F2000340421A6072
:10280C007047C04640F2D812C2F2000203001068B2
:10281C0010B1C3181360704740F2DC10C2F2000014
:10282C00F7E7C0469E2110B5C905041CFDF78CFCCA
:10283C0018B9201C00F024FC10BD9E21201CC905D9
:10284C0000F05AFA00F01CFC80231B069C466044E6
:10285C00F2E7C046F0B546464F46D646C0B54700EF
:10286C004502C30F3F0E98460E1C6D0A002F56D022
:10287C00FF2F21D0802340F2000940F2000AED0026
:10288C00DB041D437F3F730074021B0E640AF60FBA
:10289C0003B3FF2B4AD080220020E400D20414435F
:1028AC007F3B4246FF1A4B4672400F2B00D9AAE0E1
:1028BC006E499B00CB589F46002D59D17300740272
:1028CC001B0E40F20809FF2740F2020A640AF60FB9
:1028DC00002BDED174BB012342464946724019439A
:1028EC000E2904D86248890041588F464246FF2081
:1028FC000024C0052043D2071043E0BCBA46B146C1
:10290C00A846F0BD5346022BF0D0032B00D1A2E019
:10291C0042462C00012B34D100200024E9E7D5B924
:10292C0040F20409002740F2010AACE764B9022323
:10293C00FF3FD1E72000FDF711FC431F9C4076239D
:10294C005B421B1A0020ACE703234A461A4391460C
:10295C000320FC33A5E72800FDF700FC7627431F76
:10296C007F429D4040F2000940F2000A3F1A8AE77C
:10297C0040F20C09FF2740F2030A84E703286CD0CD
:10298C00320038007F30002825DD630704D00F2388
:10299C002340042B00D00434230103D53800354BDD
:1029AC0080301C40FE28A2DCA401640AC0B2A0E75F
:1029BC0080240022FF20E4039BE78023DB031D42DD
:1029CC0001D01C424BD08024E4032C4364024246C9
:1029DC00FF20640A8DE701231B1A1B2B9CDC2100B2
:1029EC009E37D940BC400B00611E8C4123435907D4
:1029FC0004D00F211940042900D00433590126D5E5
:102A0C000120002475E76D016001854213D21B2360
:102A1C000024013F0126290064006D00002901DB20
:102A2C00A84201D82D1A3443013B002BF3D16B1E65
:102A3C009D412C43A5E71A2301242D1AEAE7981E81
:102A4C0043425841404232000024C0B251E79B013E
:102A5C0000205C0A4DE746462C008023DB031C4318
:102A6C0064023200FF20640A43E7C0465C3300086E
:102A7C009C330008FFFFFFF7F0B54F464646D6469D
:102A8C00C0B546004502360E0F1C6D0AC40F002E51
:102A9C0000D1C4E0FF2E79D0802340F2000940F22F
:102AAC00000AED00DB041D437F3E7B025B0A984667
:102ABC007B001B0EFF0F002B78D0FF2B00D195E075
:102ACC0042468021D200C9041143884600217F3B35
:102ADC00F6184B46721C0A2B74DC4B467C40022BBE
:102AEC0000DCA6E048460123834040F230501842F7
:102AFC0068D140F24020184200D0ECE0B938FF38E1
:102B0C00184200D0DAE04FF6FF714746280C4346D6
:102B1C000D4039400F001B0C6F4341435D4358433C
:102B2C006D183B0C5B19994203D9802149028C46E4
:102B3C0060444FF6FF7519043D4049198D016F1E15
:102B4C00BD411B0C890E1B180D439B011D431B0122
:102B5C0000D4C5E0012369081D400D4310007F30EF
:102B6C00002800DC93E06B0704D00F232B40042BD0
:102B7C0000D004352B0103D5803210005D4B1D4075
:102B8C00FE2853DCAB015B0AC0B226E0002D00D05E
:102B9C0077E07B025B0A98467B001B0E40F208092B
:102BAC00FF2640F2020AFF0F002B86D14346002B72
:102BBC0055D14A4601331A4391464B460121721CAA
:102BCC000A2B8ADD5346022B30D0032B00D17BE03D
:102BDC005346012BC2D100200023C0051843E40743
:102BEC002043E0BCBA46B146A846F0BD330042468D
:102BFC00FF33FAB3032249461143721C8946FF3254
:102C0C000A2973DD0F295DD18023DB031D425BD0C4
:102C1C0042461A4258D13C00FF201343DDE78DB9E0
:102C2C0040F20409002640F2010A3EE7FF2000238F
:102C3C00D3E7013B012B00D965E70229F6D04546C5
:102C4C008A46C5E72800FDF789FA7626431F7642A7
:102C5C009D4040F2000940F2000A361A25E7404632
:102C6C00FDF77CFA4246431F9A40361A90460021E3
:102C7C00763E2EE749460232114389461E00022158
:102C8C0027E740F20C09FF2640F2030A0DE7012367
:102C9C001B1A1B2B9FDC9E3229009540D9406A1EC3
:102CAC0095410D436B0704D00F232B40042B00D010
:102CBC0004356B0116D5012000238EE73C004546F8
:102CCC008A467FE73C0045468023DB032B435B02AF
:102CDC00FF205B0A81E780230024FF20DB037CE7D5
:102CEC0032003BE7AB0100205B0A76E71E000321B4
:102CFC007C40F7E6FFFFFFF7F0B546464F46D64659
:102D0C0043025B0AC0B59C461F00DE004B025A0A08
:102D1C00904645004A002D0EC40F120EC90F9B0998
:102D2C00FF2A25D001204140A81A8C420FD0002840
:102D3C0000DC8AE192BB002B00D19CE0421E0128F2
:102D4C0000D14FE1FF2800D19BE010002CE00028BF
:102D5C0000DC87E1002A00D182E0FF2D00D190E059
:102D6C008022D20413431B2800DCEAE001363FE04A
:102D7C002800FF388246002B54D140F20109484606
:102D8C0041408C4200D1C4E05046002800D187E07D
:102D9C000C00002D4CD0FF2000273AE0FF2D00D175
:102DAC006FE08022D204134301221B2807DC202170
:102DBC00091A1A008B40C240591E8B411A43B61A8D
:102DCC0073016AD5B601B7093800FDF7C7F90538A4
:102DDC008740854200DD7EE020223B00401B013015
:102DEC00121A3E009340C6405A1E934100251E43C2
:102DFC00730704D00F233340042B00D00436730127
:102E0C003AD5681CFE2DC6D09B4BC0B233409B01FB
:102E1C005F0AC0053843E4072043E0BCBA46B1461C
:102E2C00A846F0BD8C4264D0D0B3002D00D0A3E0F6
:102E3C00FF20F6B1471E012800D1E1E00C00FF286D
:102E4C0000D1CDE001211B2F07DC2020C01B31005D
:102E5C008640F940701E8641314315005E1AAFE77B
:102E6C004BB1421E012800D1A0E0FF2809D0100070
:102E7C0079E70C001E000500F3089C46FF2D00D0DE
:102E8C009BE06346002B00D185E780276346FF0358
:102E9C001F437F02FF207F0ABBE77307AAD1EBE732
:102EAC00FE206A1C10421AD1002D77D1002E00D1C1
:102EBC00AAE00020002BACD08022F71AD2041742D3
:102ECC0000D1BBE001249B1B0C4013429FD06A4AEB
:102EDC00013013409BE7684E2D1A3E4088E7F71AE5
:102EEC007A0157D4002F00D06EE700240020002771
:102EFC008FE780B1002D73D1FF20002EBAD0411E78
:102F0C00012853D0FF286BD01B296EDD15005E1CE9
:102F1C006EE7514659BBFE216A1C114233D1002D7C
:102F2C0050D1002E00D186E00020002B00D170E79C
:102F3C00F318DF087F027F0A5B0100D469E70120E8
:102F4C0067E72021091A1A008B40C240591E8B4199
:102F5C001343F6187301A0D50135FF2D00D11AE7E4
:102F6C000123464A3340760816401E4340E7002DA5
:102F7C0000D010E7FF20C0E70C00C44681E7FE211B
:102F8C006A1C0A42CDD0FF2A00D104E7F6181500BE
:102F9C0076082DE701249F1B0C4015E7E6BB002BA0
:102FAC0045D180270024FF20FF0332E7F6180225C5
:102FBC007301D5D4F3089C46012563465F027F0A52
:102FCC00E8B226E766B1002B00D15EE78023DB0375
:102FDC009C4500D259E7984500D356E7C44654E7C0
:102FEC00C4464EE70125F61AEAE630002025C84013
:102FFC00691A8E40711E8E4106431500F618A9E71A
:10300C000C0001259E1BDBE6002B00D16DE7012493
:10301C00474600200C40FCE6002B00D135E780230E
:10302C00DB039C4500D230E7984500D32DE7012403
:10303C00C4460C4029E747460020EAE617B1BF0119
:10304C007F0AE6E600240027E3E6002800D127E704
:10305C00571B3800002D00D1EBE68020C0040C007B
:10306C000643EFE600288AD0511B0DB9080044E74F
:10307C008020C004064347E7FFFFFFFBFFFFFF7DF7
:10308C0041024200C30F490A0020120E7E2A03DDC2
:10309C009D2A02DD094A98187047802000040143DC
:1030AC00952A07DC9620821AD1404842002BF3D196
:1030BC000800F1E7963A9140F7E7C046FFFFFF7F23
:1030CC0070B5040070B1FDF749F803009E20C01ADA
:1030DC0096280CDC082B2DD0083B9C406402640A1B
:1030EC00C0B201E000200024C005204370BD992827
:1030FC0014DC5A1F9440220010490A40650709D07D
:10310C000F252C40042C05D00432540102D59F20ED
:10311C000A40C01A9201540AC0B2E5E71A00210015
:10312C001B3291400A00511E8A410521C91ACC401C
:10313C001443E0E764029620640AD5E7FFFFFFFB27
:10314C0070B542004E024C0045026D0A120EC30FC0
:10315C00760A240EC90FFF2A0FD0FF2C0BD00120AA
:10316C00A24209D1B54207D18B420FD022B9280017
:10317C00431E984100E0012070BD0120FF2CFBD1C3
:10318C003543002DF8D14B401800F5E70020F3E74C
:10319C0030B5420044024D02C30F4800640A120EBF
:1031AC006D0A000EC90FFF2A12D0FF2807D0B2B942
:1031BC0038B90DB3002C2AD14800013830BD1DBBE5
:1031CC000AB9002CF8D08B4205D158000138F5E72C
:1031DC00D4B9FF2813D001205B421843EEE7002836
:1031EC00F9D08B42F7D18242F5DCEEDBAC42F2D85F
:1031FC000020AC42E2D2E8E7002CDFD0EBE71DB9AF
:10320C008B42E8D10020D9E702204042D6E78B421E
:10321C00ECD0E0E730B5420044024D02C30F480049
:10322C00640A120E6D0A000EC90FFF2A12D0FF2875
:10323C0006D0AAB930B915B344BB480001380EE02A
:10324C0065B90AB9002CF8D08B4215D001205B422D
:10325C00184304E014B9FF28F8D19DB1022030BD09
:10326C000028F3D08B42F1D18242EFDC04DBAC427C
:10327C00ECD80020AC42F2D258000138EFE7002C19
:10328C00EDD0E3E700208B42E9D0DFE78B42EED0B4
:10329C00DCE7C046F8B5C046F8BC08BC9E46704793
:0C32AC00F8B5C046F8BC08BC9E46704750
:1032B80000000000000000000102030406070809DE
:1032C800000000000102030444697374616E6365C1
:1032D8003A20256409004F7665722052616E676551
:1032E8000900584C53572D3344502D556C74726156
:1032F800536F6E696320416E616C6F6720333030A5
:103308004B210D006361705F76616C3A256C64092E
:103318000054656D703A25640A006572720D0023C9
:103328002D302B2000686C4C0065666745464700C9
:1033380030313233343536373839414243444546E3
:103348000030313233343536373839616263646579
:1033580066000000122A0008FA280008242900083C
:103368008829000824290008BC2900082429000805
:1033780088290008FA280008FA280008BC2900084B
:1033880088290008102900081029000810290008B9
:10339800C6290008FA280008FA2800082429000885
:1033A8004A2A000824290008BC2900082429000802
:1033B8004A2A0008FA280008FA280008BC29000848
:1033C8004A2A0008102900081029000810290008B6
:0433D80025020008C2
:0433DC00F5010008EF
:1033E00000A24A0400000000030000008C0000203E
:1033F00014000020000000008C000020F4000020D9
:103400005C0100200000000000000000000000003F
:1034100000000000000000000000000000000000AC
:10342000000000000000000000000000000000009C
:10343000000000000000000000000000000000008C
:040000050800183D9A
:00000001FF
